:020000020000FC
:1000000055CEBCC10000000020C000008EC0000022
:10001000000098C000000000000000000203040679
:10002000080C10182030406080000406080C1018DE
:100030002030406080A0C0000003070F1F000D0D9E
:100040000403060D0503030202004FB662FD0CC057
:10005000552041F00994C52DC095089483FDC7959E
:10006000C4BD64604FBE1895C0916400089483FDC0
:10007000C795C4BD6B7FC0916400CF3F09F41EC01B
:1000800070FF1AC082FD05C04FBE9598AC98C0980D
:10009000189576FD0EC065FD0CC0C091B100C0FD85
:1000A0009498C1FDAD98C2FDAB98CAEFC095CA95B2
:1000B000F1F79598AC98C0984FBE189524BCCC2702
:1000C000C064C8BF6460F8CFC6CF70FFC4CF65FD01
:1000D000C2CF959AC0CF70FFBECF65FDBCCFAC9AA2
:1000E000BACF70FFB8CF65FDB6CFC09AB4CF949A9F
:1000F00070FFB1CF65FDAFCFC7E0CA95F1F7959A14
:10010000AACFAD9A70FFA7CF65FDA5CFC7E0CA956E
:10011000F1F7AC9AA0CFAB9A70FF9DCF65FD9BCF56
:10012000C7E0CA95F1F7C09A96CF4FB6C9B7CF7E50
:10013000C9BF6E7FCCB5CE0DDDB5DF1DDBBDCABD41
:100140004FBE18953FB68F7EABB7A074A2118061E9
:10015000A0E0ABBFA9B7AE7FA9BF7894A09168001B
:10016000AA2341F085FD2AC0A0916800AA95A0931A
:10017000680024C040E050E085FD14C0A0B396FDA7
:10018000A095A2FD4FEFA3E096FDA2E0A5BFAA2790
:10019000A064AABF8D7FA0B396FDA095A2FD5FEFDE
:1001A000451741F7A0E461FDA093680085FD03C0F9
:1001B000A0E4A093680040939600816085FD0EC086
:1001C000A0916900AA2331F0A0916900AA95A0939B
:1001D000690004C08061AA27A064AABF80FF0AC08A
:1001E000A09196004A2F61FF8E7F85FD01C000C05F
:1001F000409361004091B400443009F004C0A091E4
:100200006100A0936300A52DA03408F06860A09160
:100210006000A395A093600051F0F894A9B7A16085
:10022000A9BF84FF02C0A0E4ABBF3FBE1895A09158
:100230007400A395A093740042E050916800552388
:1002400029F085FF03C05A9550936800A09196004D
:10025000A13018F0209299000DC020929A002092AF
:10026000A300A0919900AF5FA093990018F0AFEFA1
:10027000A0939900B09061005091B400523049F4BD
:1002800066FF91F0A2E3BA1678F0A0918600A093E1
:100290006100533049F466FF39F0A2E3BA1620F04A
:1002A000A091C000A0936100509162005B1521F005
:1002B00010F05A9501C05395509362004A95D1F6BB
:1002C0005091A300539509F45A955093A300A0911F
:1002D000A400AA95A093A40009F046C0A1E0A093B1
:1002E000A40045E0A091A5005A17F0F1A091A60046
:1002F0005A1728F441E0A3E0A093A40007C0A091FE
:10030000A7005A1718F441E04093A400D0909C0035
:10031000C0906300DC14A8F0A091B400A430D9F020
:1003200066FD0FC0C0929C00539511F0A091A500EE
:10033000A093A300A1E0A093A400ACE3A09362006B
:1003400013C0A0919C00A40F20F45FEF50939C0079
:1003500002C0A0939C00A0919C00AF3F29F4AFEF96
:10036000A0939A00A093A300F894A9B7A160A9BF95
:1003700084FF02C0A0E4ABBF3FBE18953FB64CB5AA
:100380005DB58F7EABB7A074A2118061A0E0ABBF5A
:10039000A9B7AE7FA9BF789481FD23C0A2E096FDE6
:1003A000A3E0A5BF8260A0B396FDA095A2FF05C003
:1003B00040936500509366001CC1A3E096FDA2E047
:1003C000A5BFAA27A064AABF8D7F85FF01C004C175
:1003D00040E0A0B396FDA095A2FDFEC0409396001C
:1003E000EDC0A3E096FDA2E0A5BF8D7F61FF71C0C7
:1003F000A2E096FDA3E0A5BFAA27A064AABF8260E1
:100400004093910050939200A0908F004A19B090B1
:1004100090005B09BB24A22C4C38520518F42092A2
:10042000950049C0A091D400AA2359F1483C520537
:1004300028F4A0E1BA2EAAE0AA2E23C04836A1E0F3
:100440005A0728F4A8E0BA2EAFE0AA2E1AC0403D01
:10045000A2E05A0728F4A4E0BA2EAEE1AA2E11C0F9
:10046000403AA5E05A0728F4A2E0BA2EACE3AA2E3F
:1004700008C04839A8E05A0720F4A1E0BA2EA8E73E
:10048000AA2EC42EA0919300CA1AD52EA091940032
:10049000DA0ADD202AF4AFEFC094D094CA1ADA0A3F
:1004A00020929500A8E0A210A0E0CA14DA0618F481
:1004B000A1E0A09395004093930050939400409145
:1004C00091005091920040938F005093900042E031
:1004D00075C0A09165004A1BA09166005A0B94FD5F
:1004E00060C093FD5EC092FD5AC086FF03C0D52E4A
:1004F000C42E0CC05695479591FD51C05695479511
:1005000090FD4DC0D52EC42ED694C79461FD19C060
:10051000AC2DAC51AD2DA24008F005C0DD2089F412
:10052000AC2DA85C70F4A0916700A395AA2311F0EC
:10053000A0936700AA3008F44FC020929600816013
:100540004BC0A0916700AA2319F0AA95A093670059
:10055000A22C5091BA0097FD02C0A090C800AAEF4B
:10056000AA0EA22DA21DCA18DA0A4FB74170442361
:1005700019F040E050E015C0AFEFCA16D20418F0F1
:100580004FEF50E00EC0A091AC00CA9E412D000C70
:10059000441F50E008F012C04FEF50E00FC05695D6
:1005A000479594FF07C0552309F04FEFA42FA69558
:1005B0004A0F521D4F3F520508F04FEF40939600EF
:1005C000816061FF09C0AFE1A095A923AB299A2FF3
:1005D0008F7DBB2009F48062A0E4A093680085FFB2
:1005E00003C0AAE0A093680061FD03C085FD01C0BF
:1005F0008F7E85FD03C0A0E2A0936900F894A9B79F
:10060000A160A9BF84FF02C0A0E4ABBF3FBE1895A4
:1006100011E00AC013E008C01AE006C01EE104C0E1
:1006200014E602C018EC00C005E1BB27BA95F1F74B
:100630000A95D9F71A95C1F708952AE338E709C052
:1006400020E33CE806C02AE234EB03C025E238ECA4
:1006500000C012E0BB27AD9ABA95F1F7AC9ABA95F3
:10066000F1F7AC98BA95F1F7AD98BA95F1F7123069
:1006700009F0959A123009F4C09AB091AD00BA957C
:10068000F1F7123009F09598123009F4C098B7E8E4
:10069000BA95F1F71A95F1F6022FB22FBA95F1F744
:1006A0000A95D9F73A95A9F6AD9A0895221B39E033
:1006B000001F3A9509F40895221F211B18F4210FF9
:1006C0008894F6CF0894F4CF622C722CB0E0889412
:1006D000B395221F331FE0F7379527958894912E05
:1006E000802E020B130B10F4192D082D10F4889492
:1006F00001C00894661C771CBA9571F7172D062D5A
:100700000895322D11232AF43A9500951095031B74
:10071000130BF894029F712C002D129F912C802CAA
:100720007894780C172D921C292DB4E06B2E269509
:10073000179507956A94D9F7332321F00095109502
:10074000031B130B08950091B400043009F474C026
:10075000B0919600B95198F0B72FB67081F466FD4C
:100760002BC005E09090C600B92DBA9521F00AE0A3
:10077000BA9509F002E1B0917B00B01BE0F066FF92
:100780000AC0B0919E00B0939C00BFEFB093A3004D
:10079000B1E0B093A400B0916100B09363002092E7
:1007A0007E0020927F002092800020928100209283
:1007B00082006F7B41C060649090C600B92DBA95ED
:1007C00079F4B0916200B095BB1FBB1F1B2FB7958A
:1007D0000B2FB12FB170B3951B2FB02FBE7F25C04B
:1007E000B92DBA95BA9581F4B0916200B095BB1F4E
:1007F000BB1FBB1F1B2FB7950B2FB12FB370B3952A
:100800001B2FB02FBC7F14C0B0916200B095BB1FEE
:10081000BB1FBB1FBB1F1B2FB7950B2FB12FB77073
:10082000B395B3951B2FB02FB87FB0540B2F12097F
:1008300000937E0010937F00089510917B00169521
:1008400000917A000795B0917E00B01B0B2FB091FC
:100850007F00B10B1B2F28F40038BFEF1B0740F0BF
:1008600009C00F37120508F405C00FE710E002C0F9
:1008700000E81FEF00938300109384000895009117
:100880008300B09180000B0F10918400B091810023
:100890001B1F20E03091840033230AF42A95B09185
:1008A00082002B1F1AF4203F40F00AC02F3008F4BA
:1008B00007C00FEF1FEF2FE003C000E010E020EFB4
:1008C00030916300B0919B003B1718F4323030F048
:1008D00009C0B0918400BB235AF004C0B0918400D9
:1008E000BB2332F400938000109381002093820098
:1008F00008952091D70000918300000F109184008B
:10090000111FFFDE11232AF40038BFEF1B0740F050
:1009100009C00F37120508F405C00FE710E002C048
:1009200000E81FEF002352F0B0916200B01B0B2FC4
:1009300018F0013008F00AC001E008C000950F5F10
:10094000B09162000B0F08F001C00FEF009385001B
:1009500008952091D8000091810010918200D1DE8D
:1009600011232AF40130BFEF1B0740F009C00F3FED
:10097000120508F405C00FEF10E002C001E01FEF00
:10098000112352F0B0918500B01B0B2F18F00130ED
:1009900008F00AC001E008C000950F5FB091850023
:1009A0000B0F08F001C00FEF0093630008950FEFE5
:1009B000677F71FD29C072FD09C06860B0917B003E
:1009C000BA3020F0B52DB03408F4677FB091D30071
:1009D000BB23D1F0B0917B00BB23B1F00FEF10919E
:1009E0007B0064DEF894B091730072FDB5E00B9F5C
:1009F000112D002D7894112309F00FEFB0919E0076
:100A00000B1710F400919E0000939D000895009133
:100A10007A0010917B0000541140B0919D0010F4B9
:100A2000BA9501C0B39511F0B0939D000895E2D33B
:100A3000B2E074FDB1E0B7B9B6B1B068B064B6B9B0
:100A4000E7DDB2E074FDB1E0B7B9B6B1B068B0644B
:100A5000B6B9B6B1B6FDFDCF04B115B1B6B1BF7729
:100A6000B6B91FD424E72093A800222309F441C07B
:100A700030E03093A900732E7694622E6694620E55
:100A8000731E262D372D0217130778F08090A800CB
:100A9000B4E7B80DB093A8008090A900B0E0B81DED
:100AA000B093A900260D371DEECF8090A80090903E
:100AB000A9001091A90016950091A8000795169518
:100AC000079523E0169507952A95E1F72091B50043
:100AD0002A9529F42092A8002092A9000AC02A95FC
:100AE00021F0800E911E2A95E1F78092A800909245
:100AF000A90008952091B500B6B1B6FDFBCF04B1B1
:100B000015B1B6B1BF77B6B9B091AA00B395B0939D
:100B1000AA00B83060F12092AA00B091D200BB23A5
:100B200021F1112329F0B091AB00BF3F61F009C062
:100B3000B091AB000B1739F020F4BB2321F0BA952C
:100B400002C0B395E1F300919B00B093AB00BC3BB6
:100B500050F400ECBE3A38F400E8B03A20F400E477
:100B6000B23908F400E000939B007F7E08952130A5
:100B7000B1F00F3FB3E01B0790F4B4E7BB2379F06B
:100B8000B091A8000B17B091A9001B0740F4B091D9
:100B90009B00BB2359F0BA95B0939B0007C0B0915E
:100BA0009B00BF3F19F0B395B0939B0000919B0051
:100BB000B0916300B01B10F400916300B0919C00F1
:100BC0000B1750F000919C00B0919C00BF3F21F0AA
:100BD000B0919C00B0939B00502E00936400B091A4
:100BE000AA00B73009F47061089502E3F894B09157
:100BF000D9000B9F012D000C001F7894B0919B0031
:100C00000B1710F000919B000093610000936300AC
:100C1000502E0093640000939E00089520927A0065
:100C2000B0EFB0937B000895F8940CB51DB52091FA
:100C30007400789430917500609076000093750090
:100C400010937600031B160971FD03C077FD7DC06C
:100C500027C070907700209377002709222311F096
:100C60000FEF1FEF8090780090907900309378001C
:100C700060927900009175001091760008191909A9
:100C800020917A0030917B0036952795020F131F33
:100C900010F40FEF1FEF00937A0010937B0029C030
:100CA00020917A0030917B003901B4E08B2EB2E0C4
:100CB0009B2E343010F08A949A94383010F08A9435
:100CC0009A94769467948A94E1F7261937099920C3
:100CD00021F0169507959A94E1F7200F311F209384
:100CE0007A0030937B0028F43FEF30937A00309302
:100CF0007B00323008F4706871FF02C0B3E00DC0B1
:100D0000B091C40000917100023838F0B395003AF8
:100D100008F0B395B63008F0B5E09B2EB4E08B2E0A
:100D200010917B0000917A0024E0169507952A9592
:100D3000E1F70819120928F0B02FB250B12FB2090B
:100D400010F402E010E0980126C020917A00309162
:100D50007B003901769467946694669466942619AC
:100D6000320906950695200F321D20937A003093A4
:100D70007B00323008F07F7704E036952795369572
:100D8000279526952695201B10F0223008F422E0A6
:100D900089019090C40060FDFECFE0908B00F09040
:100DA0008C006160B9B7B061B9BF380177FD41C04F
:100DB0007694679400938B0010938C00B92DB33018
:100DC000E1F0B0FD04C0060D171D930106C0000F31
:100DD000111F0250120922E030E0B92DB33068F043
:100DE00020938D0030938E0000938700109388002D
:100DF0006092890070928A003AC000938D0010932F
:100E00008E00209387003093880060928900709252
:100E10008A0071FF0DC0BFE0B0938D0020928E005C
:100E2000B093890020928A00B0938B0020928C00AE
:100E30001EC0669400938B00B92DB33091F0B0FDC5
:100E400003C0060D262D03C0000F025022E0B92D6D
:100E5000B33038F020938D000093870060928900B2
:100E600006C000938D002093870060928900009156
:100E70007C0002FD0350013029F495FD0AC0B6E064
:100E8000B7B909C0023019F4B7E0B7B904C095FD8D
:100E9000F6CFB0E0B7B90091A200000F10F4BBE6A6
:100EA0000B270093A20060FDFECFB2E0B0936E006E
:100EB0006160B9B7B061B9BFB72FB670D1F02091FA
:100EC0007A0030917B00369527953695279571FFEE
:100ED00002C0B0E43B0FF8940CB51DB5020F131F10
:100EE0001BBD0ABD6160B0E1B8BFB9B7B061B9BFA1
:100EF00078940895606120927D0020E067FD20E2F3
:100F000006C0606120927D0020E267FD20E001E0E4
:100F100011E077FD11C0B72FB67009F06F7E14E1B4
:100F200000917B00069509F403950F3008F00FE05F
:100F300071FF02C004E114E160FD0FC0B0917D00BB
:100F4000BB2359F071FF06C0B0916E00BA95B09303
:100F50006E0011F4706247C0ABDFB0B7B77FB0BFAF
:100F6000B8B1B0B7B860B0BFB0917D00B395B093E1
:100F70007D00B8B177FD06C0B1E071FDB3E0BA9570
:100F8000F1F7B8B1B072B21709F022C071FF05C015
:100F90000395011708F00A95CFCF64FD05C00395AE
:100FA000011708F0B4CFC8CF6F7EF8943CB56DB48C
:100FB00070907A0080907B00370D681C6BBC3ABD46
:100FC0006160B0E1B8BFB9B7B061B9BF78949FCFE5
:100FD000B0916D00B13008F49ACF64FD98CF0A95B6
:100FE00009F0AACF7F7D20918D0030918E00F8947A
:100FF000B0E1B8BF0CB51DB5020F131F1BBD0ABD74
:10100000E0908700F09088006160B9B7B061B9BF27
:101010007894B72FB67039F0B0916D0072FFB39528
:10102000B0936D0009C075FF07C067FD05C064FD82
:1010300003C0BF91BF91E5C4089500E063FF03C002
:1010400064FF01C001E0F89410917100B7E01B9FAC
:10105000212D102D7894200F2695179526951795FC
:101060002695179510937100183718F4B8E7B093C8
:10107000710000917100B09172000B1720F0606256
:101080009598AC98C09860FDFECFE0908900F090F4
:101090008A006160B9B7B061B9BF0895B2E095FD4B
:1010A0000AC0F894B0937C00AD9A949862FF01C096
:1010B000C09A7894F4C0F894B0937C00AD9AAB9841
:1010C00062FF01C0959A7894EAC0B3E082FF24C021
:1010D00095FD11C002E0F894B0937C00E1E8F0E0E7
:1010E0000093B100C098AB9A62FF02C0AC9A01C0F5
:1010F000AD987894D4C002E0F894B0937C00E1E815
:10110000F0E00093B1009598949A62FF02C0AC9A07
:1011100001C0AD987894C3C095FD0BC0F894B0930E
:101120007C00EBE6F0E0C09862FF01C0AC9A7894D6
:10113000B6C0F894B0937C00EBE6F0E0959862FFBF
:1011400001C0AC9A7894ABC0B4E095FD0AC0F894A5
:10115000B0937C00949AAB9862FF01C0AC9A7894EB
:101160009EC0F894B0937C00AB9A949862FF01C043
:10117000AC9A789494C0B5E082FF24C095FD11C06C
:1011800001E0F894B0937C00E7E7F0E00093B10051
:10119000AC98AD9A62FF02C0959A01C09498789479
:1011A0007EC004E0F894B0937C00EBE8F0E000939C
:1011B000B100AC98AD9A62FF02C0C09A01C0AB9872
:1011C00078946DC095FD0BC0F894B0937C00E5E673
:1011D000F0E0AC9862FF01C0959A789460C0F894F2
:1011E000B0937C00E1E7F0E0AC9862FF01C0C09AE8
:1011F000789455C0B6E095FD0AC0F894B0937C0091
:10120000AB9AAD9862FF01C0959A789448C0F89463
:10121000B0937C00949AAD9862FF01C0C09A789414
:101220003EC0B1E082FF24C095FD11C004E0F894F7
:10123000B0937C00EBE8F0E00093B1009598949AAD
:1012400062FF02C0C09A01C0AB98789428C001E048
:10125000F894B0937C00E7E7F0E00093B100C09809
:10126000AB9A62FF02C0959A01C09498789417C017
:1012700095FD0BC0F894B0937C00E1E7F0E0959801
:1012800062FF01C0C09A78940AC0F894B0937C00C1
:10129000E5E6F0E0C09862FF01C0959A78946F7D12
:1012A000089524E630E0F9012092B1009598AC98B9
:1012B000C098949AAD9AAB9A6B7F0895A2EBB0E078
:1012C00007E00D9307E00D9301E00D9304E00D930B
:1012D0000FEF0D930D9309E00D9302E00D9301E0E4
:1012E0000D9301E00D93AEEBB0E001E00D9300E053
:1012F0000D9304EB0D930FEF0D930D930D9303E0FE
:101300000D930FEF0D9301E00D930FEF0D9305E299
:101310000D9300ED0D9308E70D9308EC0D9304E099
:101320000D930FEF0D9301E00D9300E00D930AE78D
:101330000D930AE00D9300E00D9301E00D9300E0A2
:101340000D930FEF0D9300E00D9308952091B900D8
:101350008B7F233009F48460B091BA009F7DB1FD8A
:1013600090629F7BB091BB00B1FD9064223011F080
:10137000886001C0877F08950A95E00FF21DB4913F
:101380000895ECE1F0E00091B200F6DFB093D700F1
:10139000ECE1F0E00091B300EFDFB093D800EAE2B7
:1013A000F0E00091B800E8DFB093D9000091D100DF
:1013B000002309F40395013108F001E1B02FB00FCB
:1013C000B00FB093A5001B2FB10FB10FB00FB093AA
:1013D000A600B10FB00FB00FB093A7000091B800F6
:1013E000023008F402E000937300B091CE000FEFDA
:1013F000B23009F400EAB33009F402E80093720055
:10140000E8E3F0E00091D500B7DFB093A0000895C5
:1014100008952091C8003091C900B091BA00B3304E
:1014200009F43E5097FF02C020E03FEFB32FB21BFC
:101430006B2EB25810F4B2E86B2E00E00395609E5C
:10144000B12DBD57D8F30093AC0008959068E1DF4B
:10145000E5D820E030E0B0E16B2EDCD8B09196000A
:101460002B0F321D6A94C9F7B4E036952795BA95CB
:10147000E1F7822E9F77CDDF0895F894E3E0F0E066
:10148000B9E0B7BFB491B078C1F3F894A895B1B5FD
:10149000B861B1BDB0E0B1BDB4E0BEBFBFE5BDBF96
:1014A00000DFB0E0B8BBB1E1B7BBB8E2B5BBB8E3B1
:1014B000B4BBB0E1B2BBB0E3B1BB2224A0E0B0E06A
:1014C0002D92AA31E9F7A0E6B0E00FEF2D920A9530
:1014D000E9F7B1E0B093A200F1DED0D2B6B1B460CA
:1014E000B6B90091CA000093AD00B1E0B0936A00B4
:1014F000F89498D8A2D892D8A3D890D8A4D88ED847
:101500004CD390D88FD88CD8F8940AEF1AEFA0B3A8
:1015100096FDA095A2FF1FC01A95C9F70A95B1F7CD
:10152000E0E0FCE1B591B43E39F4B591B03E21F470
:10153000B591BF3F09F40CC0E0E0F395F395B59188
:10154000B83F49F4B591B43931F4B591BA3A19F4C8
:10155000EE27F6950994FADE14DF5ADF5ADF009180
:10156000CA000093AD009DDEB2E0B3BFB2E0BEBDE5
:10157000B2E0B5BDB1E5B8BFB9BFB0B7B77FB0BFD6
:10158000B8B1B0B7B860B0BF43D8789450DA209201
:101590007000B3E096FDB2E0B5BFB0E4BBBFBB27BF
:1015A000B064BABF8D7F3ED8626033E02CE0B0916A
:1015B0009500BB2321F42CE03A9509F4A5CF2ED851
:1015C00080FFA2CF8E7FB0919600B23078F3B92F12
:1015D000BF710091980000939700B0939800B017E6
:1015E00029F72A9521F76D7FB3E096FDB2E0B5BFEC
:1015F000BB27B064BABF8D7FB091D400BB2321F468
:101600008062B92FB0709B2F8F7B2092670008D823
:1016100085FF05C0B0916700BA3008F08064FAD742
:1016200002E085FF01C000E0B0919600B017B8F36A
:10163000F89403D802D801D87894F4D72092860081
:10164000E9D7B091BE00B13008F46EC0B0916A0025
:10165000B13008F469C085FD18C0B0919600BF3F55
:1016600008F462C0F894F2D77894DAD7B091960073
:10167000B130C0F7F894E1D7CFD7DFD77894D0D77F
:10168000B0919600BF3FB0F3BAC2B8E09B2E90680D
:10169000F894BFDE7894C4D7F8949F77BADE809030
:1016A0009600B0919600BF37789408F445C0B0D743
:1016B000F894CCD778949A9451F7C8DEB82DB550E9
:1016C000B093C900AFD7F89406D26CD27894BAE040
:1016D0009B2E9068F8949DDE7894A2D7F8949F771B
:1016E00098DE80909600B0919600BF37789478F796
:1016F0008FD7F894A2D790D7A0D778949A9449F727
:10170000A5DEB82DBB5FB093C8008CD7F894E3D1A9
:1017100058D2789485D7F8947CDE7894B09196006E
:10172000BF3F08F498CF6BC200919600B09186003D
:101730000B1710F00093860073D701E0B091BA0048
:10174000B35009F405E0B0919600B01708F078CFD7
:10175000F8947CD77BD77AD7789464D720926A00A4
:1017600020926B0020926C00B0916B00B395B09307
:101770006B00BF3F71F5B0916C00B395B0936C00F6
:10178000B091CC0009E1BA9559F002E3BA9541F065
:101790000DE7BA9529F00AEFBA9511F020926C0086
:1017A000B0916C00B017A8F07CDD32D7B0916C001E
:1017B000BA95B0936C0020926B00B091CB00B093BF
:1017C000AD00F89443D77894B091CA00B093AD00BF
:1017D00027D722D7B0916800BB2319F485FF01C039
:1017E00093CE01E085FD01C006E0B0919600B017F0
:1017F00008F4BACF15D7B0916800BB2309F484CEA2
:10180000F8944FDD209261002092620020926300E4
:10181000522C209264002092A1007894B091B700DD
:10182000BB0FB0939F0020927E0020927F002092F9
:10183000800020928100209282002092AA0060E025
:1018400070E020927100B8E0B093AA007061E0D619
:10185000B2E074FDB1E0B7B9B6B1B068B064B6B982
:10186000B6B1B6FDFDCF04B115B1B6B1BF77B6B90B
:10187000112309F00FEF0093AB003CD9B8E0B0930F
:10188000AA00706163DDF894BFEFB0939B00ADD9FF
:10189000B0916100B0939B00B0939C00B0939D0009
:1018A0007894B1E0B0936100B09363005B2EB09385
:1018B0006400B093A400B0919A00B093A300B091DB
:1018C000BA00B33019F49F7D87FD90627160726039
:1018D00020926D008FDCA5DCA1D9A6D99FD9A4D90F
:1018E0009DD90FDB30D7A9DBD9DB9ED903DB66FDA1
:1018F000A4D777FF5CD877FD8AD89FDBE6DB94D945
:1019000000DB66FDBCD799DB1FDC8ED9F3DA66FD00
:10191000F0D793DB30DC88D9F4DA66FD1AD88DDB9A
:1019200069DC82D9E7DAB2E074FDB1E0B7B9B6B1EB
:10193000B068B064B6B981DB74DC76D9DBD871FFEE
:101940001EC0B0919E00B0939B00B0939C00B091DC
:101950009A00B093A300B1E0B093A40018E12CE08A
:10196000B0916D00B11728F07D7F746020936F00F7
:1019700006C0B0919600B13008F0B3CF4CC072FFF2
:1019800011C067FD0FC0B0916F00BA9519F47B7F4D
:101990007860A7CFB0936F00B0919600B13008F097
:1019A000A0CF39C020927000B0919900B13058F0AA
:1019B000B0919E00B0939C00B0919A00B093A300A8
:1019C000B1E0B093A400B09199000AEF1091D60055
:1019D000112309F003E0B01708F01DC085FF04C013
:1019E000B0916800BB23B9F000EF67FF05C0B0916C
:1019F0009E00B0939B0000E2B0917B00B01708F40A
:101A000070CFB0917000B395B0937000B091960014
:101A1000BB2309F002C020927000F89442DC809051
:101A2000B900B2E0B093B90091DC8092B900209285
:101A300061002092620020926300522C2092640088
:101A400020929F0060E070E07894EAD52ADC009153
:101A5000D600002319F0959AAC9AC09AB6B1B4603A
:101A6000B6B985FF05C0B0916800BB2309F44CCD21
:101A7000B091BF00B13008F0D2CD72CEEDE0F0E011
:101A800023D0053A09F01BC0EEE0F0E01DD00A3586
:101A900009F015C03AE0A2EBB0E0E3E0F0E014D0CA
:101AA0000D9331963A95D9F739E1AEEBB0E0EFE01E
:101AB000F0E00AD00D9331963A95D9F702C0FEDBDB
:101AC0000AD0E8E2F0E00895E199FECFEEBBFFBB5B
:101AD000E09A0DB308951ED03AE0A2EBB0E0E3E047
:101AE000F0E00D910FD031963A95D9F739E1AEEB90
:101AF000B0E0EFE0F0E00D9105D031963A95D9F7DE
:101B000012D00895E199FECF0DBBEEBBFFBBE29A68
:101B1000E19A0895EDE0F0E00FEFF4DFEEE0F0E0A1
:101B20000FEFF0DF0895EDE0F0E005EAEBDFEEE027
:101B3000F0E00AE5E7DF08953091AE000091AF00D4
:101B4000313011F40093B200323011F40093B3003D
:101B5000333011F40093B400343011F40093C60014
:101B6000353011F40093B500363011F40093B8000D
:101B7000373011F40093C400383011F40093B900E9
:101B8000393011F40093CE003A3011F40093BA00CA
:101B90003B3011F40093BB00089525E043D52A950E
:101BA000E9F708954AD54CD54ED550D535D545D50C
:101BB00047D549D54BD530D540D542D544D546D566
:101BC000089544D540D53CD538D526D53FD53BD50D
:101BD00037D533D521D53AD536D532D52ED508953A
:101BE0008090AE009090AF0028D527D526D514D58B
:101BF0008A94D1F72BD510D59A94E1F70895F894EB
:101C0000D1DF7894CADFC9DFB1E0B093AE00B1E0B4
:101C1000B093AF002092B000F894E2DF7894B5E082
:101C20006B2E70909600FED4B09196007B16C9F78B
:101C3000B13018F0BF3F40F107C07EDFF8944BDFB2
:101C4000B1DFB8E0B1BDA9DF6A9459F7B091B00037
:101C5000B395B093B000B33008F4DECF9EDFB091FF
:101C6000AF00B395B093AF00F894B091AE00BA95C1
:101C7000EEE3F0E0EB0FF21D049178940395B09140
:101C8000AF00B01708F4C6CF88DF87DFB091AE0091
:101C9000B395B093AE00B091AE00BC3008F4B7CFAE
:0E1CA0000DDBF89418DFB8E0B1BD77DFE6CBBE
:00000001FF
